:030000000232B316
:0C32B30078FFE4F6D8FD75815E0232FA67
:100E9E000A53746172743A20004950436F6E6E6546
:100EAE0063745245510A004950436F6E6E65637408
:100EBE00003E432C562C43432CC0E4E0EFF2E5F009
:100ECE0020D1E8EDEAEEEC49500A003E432C4D41AC
:100EDE00432C25303262583A25303262583A25304A
:100EEE003262583A25303262583A25303262583AD8
:100EFE0025303262582C4D414320E0E4F0E5F10AF2
:100F0E00003E432C5645522C20332E3120EEF2203B
:100F1E0025732025732CC2E5F0F1E8FF20495020FF
:100F2E00ECEEE4F3EBFF0A004E6F76203033203206
:100F3E003030370030383A35323A3138003E432CB3
:100F4E004C442C50524F473A202020202020202065
:100F5E002020202020202020202020202020202083
:100F6E002020202020202020202020202020202073
:100F7E002020202020202020202020202020202063
:100F8E00202020202020202020202020202CC4E0E3
:100F9E00F2E020EFF0EEF8E8E2EAE828F4E0E9EB20
:100FAE00290A003E2A2C312CCEF1EDEEE2EDFBE5C6
:100FBE0020EFE0F0E0ECE5F2F0FB20F1E5F2E5E207
:100FCE00EEE3EE20E8EDF2E5F0F4E5E9F1E00A00FB
:100FDE003E412C4130312C2562752E2562752E2511
:100FEE0062752E2562752C495020E0E4F0E5F12063
:100FFE00E0E4E0EFF2E5F0E00A003E412C41303251
:10100E002C2562752E2562752E2562752E2562752C
:10101E002C495020E0E4F0E5F120EEF1ED2E20F128
:10102E00E5F0E2E5F0E00A003E412C4130332C259C
:10103E0062752E2562752E2562752E2562752C49D8
:10104E005020E0E4F0E5F120F0E5E72E20F1E5F0A8
:10105E00E2E5F0E00A003E412C4130342C25627569
:10106E002E2562752E2562752E2562752CCCE0F12B
:10107E00EAE020F1E5F2E80A003E412C4130352C41
:10108E002562752E2562752E2562752E2562752CAC
:10109E00D8EBFEE70A003E532C4130362C25627504
:1010AE002CC2F0E5ECFF20EEE6E8E42E20EAE2E8C2
:1010BE00F2E0EDF6E8E820282A3130ECF1290A00BA
:1010CE003E2A2C312CC4EEEF2E20EFE0F0E0ECE5C2
:1010DE00F2F0FB20F1E5F2E5E2EEE3EE20E8EDF2D0
:1010EE00E5F0F4E5E9F1E00A003E422C5330312CF4
:1010FE002562752CC6E4E0F2FC20E7E0EFF0EEF19D
:10110E00E020F1EEE5E4E8EDE5EDE8FF20EEF2207B
:10111E00F1E5F0E2E5F0E00A003E422C5330322CCD
:10112E002562752CCEE1ECE5ED20F120F1E5F0E243
:10113E00E5F0EEEC20E1E5E720EAE2E8F2E0EDF69C
:10114E00E8E90A003E422C5330332C2562752CCF31
:10115E00E5F0E5E7E0EFF3F1EA20EFF0E820EFEE5F
:10116E00F2E5F0E520F1E2FFE7E820F120F1E5F00D
:10117E00E2E5F0EEEC0A003E422C5330342C2562B0
:10118E00752CCDE5F220EFE5F0E5E4E0F7E820E49C
:10119E00E8E0E3EDEEF1F2E8EAE820E220F1E5F036
:1011AE00E2E5F00A003E422C5330352C2562752CB8
:1011BE00CAE0EDE0EB20F8E8F0EEEAEEE2E5F8E06A
:1011CE00F2E5EBFCEDEEE3EE20EEE1ECE5EDE00A10
:1011DE00003E532C5330362C253032625825303297
:1011EE0062582530326258253032625825303262CC
:1011FE005825303262582C4D414320E0E4F0E5F1A1
:10120E0020F8E8F0EEEAEEE2E5F8E0F2E5EBFCEDD0
:10121E00EEE3EE20EEE1ECE5EDE00A003E454E4455
:10122E000A0044756D705820202020203030203068
:10123E0031203032203033203034203035203036DB
:10124E0020303720303820303920304120304220B5
:10125E0030432030442030452030460A003A2000EA
:10126E000A0044756D70442020202020303020303C
:10127E00312030322030332030342030352030369B
:10128E002030372030382030392030412030422075
:10129E0030432030442030452030460A00457272DB
:1012AE00206B657900526420656570726F6D0A005F
:1012BE005264204D454D0A00526420436F64650A06
:1012CE000044656275674950204F4E0A00446562BE
:1012DE0075674950204F46460A004465627567554A
:1012EE00736572204F6E0A004465627567557365AB
:1012FE0072204F46460A0044656275674D7367203B
:10130E004F6E0A0044656275674D7367204F4646FF
:10131E000A00436F6E666967206C6F636B210A006B
:10132E00577220656570726F6D0A00205361766585
:10133E0020656570726F6D210A00457272204D41F5
:10134E004321004C6F61643E3E002A003C41303127
:10135E003D003C4130323D003C4130333D003C418C
:10136E0030343D003C4130353D003C4130363D008F
:10137E004E4F4950004C494E4B434F4E5452005421
:10138E0052415353004652004E4F4C494E4B00496A
:10139E004E49004E4F4449414700003C21003C530A
:1013AE0030313D003C5330323D003C5330333D0034
:1013BE003C5330343D003C5330353D003C533036C9
:1013CE003D00FF137EFF1383FF138DFF1393FF1357
:0A13DE0096FF139DFF13A1FF13A853
:063C1400010B0001090094
:103C7F00C2AFC28E438910758BFF758DB7D2ABD291
:043C8F008ED2AF2200
:03001B0002318926
:10318900C0E0C083C082C0D0C2AFC28E758BFF754C
:103199008DB720060675A61E75A6E10509D202E5BA
:1031A9000B6002050BE50AD394014002150A050ECE
:1031B900E50E540F7050D20DE50E543F701AD2002F
:1031C90090668DE0601204F0E0D394B4400A9080D8
:1031D900007480F0C2AF80FE906688E0600204F05F
:1031E900906104E0600214F090668EE0D39401408F
:1031F90003E014F0300502050CE50DD39464400496
:10320900D2068002050DE508D3940140021508D2C3
:0C3219008ED2AFD0D0D082D083D0E03273
:10088100C291C290D2B5C20A7D027C007F07123BA1
:10089100F78F24E524646060097D017F60123BAF1E
:1008A100D20AE4FDFC7F0B123BF78F24E52430E6EE
:1008B100097D04E4FF123BD3D20A7D017C007F074E
:1008C100123BF78F24E5247008FD7FFF123BAFD266
:1008D1000A300A03126000C2AFC288C2A8C2AA7558
:1008E1008900123654906341E0B4FA09A3E064CE62
:1008F1007003020981E4F52474392524F582E43476
:1009010063F583E4F00524E524B443EC906341747A
:10091100FAF0A374CEF0A374CCF0906347740AF09C
:10092100E4A3F0A304F0A3F090634C7403F0A37468
:10093100CCF090633D74FFF0A3F0A3F0E4A3F0903A
:1009410063587405F0E4F524E5242401FFE433FE43
:1009510074392524F582E43463F583E0FD123C66A5
:100961000524E524C3944340DFE4F5A775A61E756D
:10097100A6E1907FF0F0A3F09080007480F080FEFB
:10098100D2AF90634C7403F0A374CCF0E490634B4A
:10099100F0122D6AEF6003122087C2B5123554C2DE
:1009A10006123A39906358E0C3940350037403F07C
:1009B100D20AC20CC20BD293200A077E0E7F9E126E
:1009C1002E50E4906578F0123C7FC2AFA37408F01A
:1009D1009062B77424F0E4A3F0906341E09062B9AF
:1009E100F0906342E09062BAF0906343E09062BBA2
:1009F100F0906344E09062BCF0906345E09062BD8A
:100A0100F0906346E09062BEF0750A01E490657A69
:100A1100F0C207C208D2AF75A70775A61E75A6E179
:100A2100200A18AF24FE7D03122F31E4FF1230DFBC
:100A31007E637F78E4FB7D0112300B90668DE06070
:100A4100037401F0E4906104F0A37455F0A3748180
:100A5100F0E4F50CE4F50D906104E07003121B5B0A
:100A610090668EE0B401119080007410F0E49066FD
:100A71008EF0D20AD20BD20C908008E0F52430E43B
:100A810005D2077410F0E52430E508D209908008FA
:100A91007420F0E52430E608D2089080087440F014
:100AA100E50CD394034023908002E4F0908001F0A0
:100AB100908000F0E50CD39406400FE4F50CC203DE
:100AC10090657AF0750A01123A399080A0E07003BE
:100AD10012374D9080B8E070031237C79080D0E094
:100AE1007003123919908000E07013300710122B37
:100AF10063906334EFF0D39400400312002690809A
:100B010002E07006908000E06005D205020A55C23D
:100B110005E4F50C906104E06003020A5530091206
:100B21001228F0906334EFF0D394004005E0FF12F7
:100B31003C97200803020CB412277B906334EFF03A
:100B41007003020A55906378E054BF247F7003025A
:100B51000C17147003020BEF24026003020C4A20ED
:100B61000A077E0E7FA7122E50300E792003769051
:100B71006350E07006906354E0605B906684E0FF30
:100B8100906350E0B50724906685E0FE906351E0E4
:100B9100B50618906686E0FE906352E0B5060C90AB
:100BA1006687E0FE906353E06E602B906354E06FC4
:100BB1007033906685E0FF906355E0B50727906636
:100BC10086E0FF906356E0B5071B906687E0FF90D3
:100BD1006357E0B5070F90657A7401F0123C9A757E
:100BE1000A01020CB490668474FFF0020CB49066A2
:100BF1008DE060037401F090667CE0FF90637AE021
:100C01006F6003020CB490667CE004F0E4F50A9096
:100C11006578F0020CB4300303020CB4906347E032
:100C21007003020A5512001ED203E4F50A9065789A
:100C3100F090668804F0E490667BF0A3F0200A73DC
:100C41007E0E7FB5122E50806A90668DE06003742F
:100C510001F0300352906378E020E74B90637AE033
:100C6100FF90667BE0FE6F600D906683E07007EE9B
:100C7100146F703F801390667BE004F0906334E062
:100C8100FFD394044003123C999060007482F0A356
:100C91007401F090637AE0906002F07E607F007DE5
:100CA100031236D2020A55300E09200306906684DB
:100CB10074FFF0200303020D69E50A706B123225FF
:100CC100EF60207E647F78906479E02404FD123621
:100CD100D2906683E06003020A55906358E0F50AFA
:100CE100020A55906688E0D3943C403C906683E0CC
:100CF100703690668804F09062B6E0702B123C98D2
:100D0100E4906478F0A37412F090667CE090647AC9
:100D1100F0A374FDF090610763A20190647C63A26B
:100D2100017F12122355809B123C93EF6015906056
:100D3100007483F0E4A3F07E607F007D021236D25E
:100D4100020A55E50A64016003020A55906578E0DC
:100D510004F0E0C394055003020CC4C203E490659F
:100D61007AF0123C9A020A55E50A64016003020A0C
:100D71005590657AE014604024FE603C14700302D3
:100D81000E5124046003020A55E4F50C200E139061
:100D9100657A7404F0906578E05401F0750A0102F7
:100DA1000A55E490657AF090657804F0750AC89068
:100DB100668474FFF0020A55906684E07003020EA7
:100DC100409064787480F090647A7401F0E4A3F048
:100DD100A304F0A37430F0A3747BF0E4F524747FD2
:100DE1002524F582E43464F583747DF07480252430
:100DF100F582E43464F583E4F0E524240790647912
:100E0100F07C667D8490634CE0FAA3E0FB7F0212E4
:100E1100344E7E647F78E5242409FD1236D2906633
:100E210083E0601B12001ED203E4F50A906578F09E
:100E310090668804F0E490667BF0A3F0020A559076
:100E4100657A7404F0906358E02432F50A020A5579
:100E51009080027410F0750A03906578E06401FFD8
:100E6100F090657A7401F0EF7019906354E06013AB
:100E7100FCA3E0FDA3E0FEA3E0FF906684121F49FE
:100E8100020A55906350E0FCA3E0FDA3E0FEA3E05D
:0C0E9100FF906684121F49020A5580FE83
:010E9D002232
:10002600906379E0B444047F0180027F0090637896
:10003600E0B447047E0180027E00EE5F604A906372
:1000460041E090637AF0906342E090637BF09063C6
:1000560043E090637CF0906344E090637DF09063AE
:1000660045E090637EF0906346E090637FF0906396
:10007600797452F09062B063A2019080A863A201E5
:100086007F06122355020877906334E0C394085024
:1000960003020880906341E0FF90637AE06F60039B
:1000A600020880906342E0FF90637BE06F6003028A
:1000B6000880906343E0FF90637CE06F6003020872
:1000C60080906344E0FF90637DE06F6003020880E8
:1000D600906345E0FF90637EE06F600302088090C6
:1000E6006346E0FF90637FE06F60030208809063E1
:1000F60079E0B444159062B0E0B4FF0E63A20190BB
:1001060080A863A2017F0612235590668DE06003E6
:100116007401F090668E7464F09063797452F09076
:100126006378E0646D60030202A37BFF7A0E79BFF9
:100136001218617BFF7A0E79D9906341E0F52EA300
:10014600E0F52FA3E0F530A3E0F531A3E0F532A307
:10015600E0F533121861752EFF752F0F7530367561
:1001660031FF75320F7533427BFF7A0F790F121804
:10017600617BFF7A0F794B1218617BFF7A0F79B199
:100186001218617BFF7A0F79DE906347E0F52EA3A4
:10019600E0F52FA3E0F530A3E0F5311218617BFFFF
:1001A6007A107908906350E0F52EA3E0F52FA3E0CE
:1001B600F530A3E0F5311218617BFF7A107936909D
:1001C6006354E0F52EA3E0F52FA3E0F530A3E0F5A8
:1001D600311218617BFF7A10796490633DE0F52E49
:1001E600A3E0F52FA3E0F530A3E0F5311218617B0B
:1001F600FF7A107987906339E0F52EA3E0F52FA3F7
:10020600E0F530A3E0F5311218617BFF7A1079A48E
:10021600906358E0F52E1218617BFF7A1079CE12A2
:1002260018617BFF7A1079F7A20EE433F52E1218C7
:10023600617BFF7A117927906683E0F52E121861AB
:100246007BFF7A11795290668DE0F52E1218617B4C
:10025600FF7A1179859062B6E0F52E1218617BFF60
:100266007A1179B3A201E433F52E1218617BFF7A75
:100276001179DF90667DE0F52EA3E0F52FA3E0F57A
:1002860030A3E0F531A3E0F532A3E0F533121861AF
:10029600122C677BFF7A12792A12186122906378F2
:1002A600E0644C70527E127F30122E50906380E0D4
:1002B600F525A3E0F526E4F5277D03AF26AE251246
:1002C6002F317E127F6B122E50AE25AF26E4FB7DBA
:1002D6001012300B7E127F6E122E5074102526F5EA
:1002E60026E43525F5250527E527C3941040CA7E63
:1002F600127F6E122E5022906378E0646C705CF56B
:10030600297E127F70122E50E4F528AF297E007DDB
:1003160003122F317E127F6B122E50E4F527A82987
:10032600E6FF74822527F582E43463F583EFF00552
:10033600290527E527B410E67E637F82E4FB7D105E
:1003460012300B7E127F6E122E500528E528C394BC
:100356000840B87E127F6E122E5022906378E064B9
:100366004B7061F527746A2527F582E43463F583BB
:10037600E06032746A2527F582E43463F583E0F49D
:100386006023746A2527F582E43463F583E0FF74FD
:10039600802527F582E43463F583E0B50710052749
:1003A600E527B408C09061047432F00208779063C0
:1003B600787421F0300A030208777E127FAB122E82
:1003C60050020877906378E0B4521A200A077E122A
:1003D6007FB3122E509063787472F07E637F787DBF
:1003E600081234D222906378E064497045200A07E7
:1003F6007E127FBE122E50906380E0F525A3E0F5B5
:1004060026E4F527852682852583E0FF7482252745
:10041600F582E43463F583EFF00526E526700205E0
:10042600250527E527B480DC7E637F787D8A123434
:10043600D222906378E064437079A3E064527046F8
:10044600200A077E127FC6122E50906380E0F525A3
:10045600A3E0F526E4F527852682852583E493FF28
:1004660074822527F582E43463F583EFF00526E5EB
:1004760026700205250527E527B480DB7E637F7895
:100486007D8A1234D222906379E0645760030208B1
:1004960080906380E0F525A3E0F52674822527F594
:1004A60082E43463AD82FC7B80AF26AE25123B55D9
:1004B600020877906378E06444600302054A90631B
:1004C60080E0FF64447003020877EFB4310CC20A7F
:1004D6007E127FCF122E50020877906380E0B430F0
:1004E6000CD20A7E127FDB122E50020877906380B0
:1004F600E0B4320CD20B7E127FE8122E500208773F
:10050600906380E0B4330CC20B7E127FF6122E503D
:10051600020877906380E0B4340CD20C7E137F051A
:10052600122E50020877906380E0B4350CC20C7E20
:10053600137F12122E50020877906380E0FF123C60
:1005460096020877906104E07013200A077E137FF5
:1005560020122E509063787421F00208779061047F
:100566007432F0906378E0FFB4510A908000748092
:10057600F0C2AF80FEEF64577045200A077E137FF6
:100586002E122E50906381E0906334F0E4F52790AC
:100596006334E0FFE527C39F400302087774822592
:1005A60027F582E43463F583E0FF906380E0252736
:1005B60024AFF582E43461F583EFF0052780D0900F
:1005C6006378E064536003020679200A077E137F8E
:1005D60039122E50906341E0FF9061B8E06F703C95
:1005E600906342E0FF9061B9E06F7030906343E042
:1005F600FF9061BAE0B50724906344E0FF9061BBC9
:10060600E0B50718906345E0FF9061BCE0B5070CC4
:10061600906346E0FF9061BDE06F6016906378746A
:1006260021F0300A030208777E137F48122E50020B
:100636000877E4F527E4F50DAF27FE74AF2527F517
:1006460082E43461F583E0FD123C660527E527C3A5
:1006560094FE40E19080007480F0C2AFE4907FF099
:10066600F0A3F0907FFD74AAF0A374FFF0A3745575
:10067600F080FE906378E0644F704C906380E0F504
:1006860025A3E0F526E5264525700A200A077E13F0
:100696007F51122E50200A077E137F58122E50E4E7
:1006A600F52774822527F582E43463F583E08526F1
:1006B60082852583F00526E526700205250527E5B2
:1006C60027B480DE020877906378E0FFB445279070
:1006D60080007480F0906380E0FDA3E0907FF0CD11
:1006E600F0A3EDF0C2AF907FFD74AAF0A374FFF003
:1006F600A37455F080FEEF6465600302087790638B
:1007060080E0FFA3E0907FF0CFF0A3EFF0E4F525C3
:10071600F526D3907FF1E09526907FF0E095254071
:1007260020E4F50D2526FFE5253401FE8526828584
:100736002583E0FD123C660526E526700205258028
:10074600D17E137F5A1233C9EF4E602012000390F8
:100756006347EFF0120003906348EFF01200039036
:100766006349EFF012000390634AEFF07E137F6057
:100776001233C9EF4E6020120003906350EFF0125F
:100786000003906351EFF0120003906352EFF012F2
:100796000003906353EFF07E137F661233C9EF4E6A
:1007A6006020120003906354EFF01200039063552B
:1007B600EFF0120003906356EFF0120003906357B8
:1007C600EFF07E137F6C1233C9EF4E6020120003E8
:1007D60090633DEFF012000390633EEFF0120003CA
:1007E60090633FEFF0120003906340EFF07E137FBB
:1007F600721233C9EF4E6020120003906339EFF096
:1008060012000390633AEFF012000390633BEFF09F
:1008160012000390633CEFF07E137F781233C9EF2A
:100826004E60081239DC906358EFF0E4F527E4F5E2
:100836000DE5272401FFE433FE74392527F582E40C
:100846003463F583E0FD123C660527E527C3944330
:1008560040DC9080007480F0C2AFE4907FF0F0A39B
:10086600F0907FFD74AAF0A374FFF0A37455F08096
:0A087600FE7E637F787D081234D205
:010880002255
:103B1D00AE07EEC39430400BEED394395005EE242E
:103B2D00D0FF22EEC39461400BEED394665005EEA8
:103B3D0024A9FF22EEC39441400BEED394465005C9
:083B4D00EE24C9FF22AF06229D
:103C4C009062AFE004F070069062AEE004F0906217
:0A3C5C00AEE0FEA3E0FF123C3022B0
:10000300123C4C123B1DEFC454F0FEC006123C4C94
:08001300123B1DD0E02FFF227B
:1039DC00E4906A68F0123C4C906A69EFF0C3943042
:1039EC004018E0FFD394395011906A68E02407F531
:1039FC0082E43461F583EFF08011906A68E024076B
:103A0C00F582E43461F583E4F0800C906A68E0049C
:103A1C00F0E0D3940840BE752D00752E00752F0074
:0C3A2C00E4F5307B017A6179071225D7A0
:013A3800226B
:0433C9008E2A8F2B8E
:1033CD009062AEE4F0A374FFF0123C4CEF606EF42B
:1033DD00606B852B82852A83E493B507EC752C01F0
:1033ED00E52B252CF582E4352AF583E493602590B1
:1033FD0062AFE0252CFF9062AEE03400FE123C304F
:10340D00E52B252CF582E4352AF583E493B50704E5
:10341D00052C80CCE52B252CF582E4352AF583E4AB
:10342D009370A6E52C24FFFFE434FFFE9062AFE01D
:10343D002FF09062AEE03EF07E007F0122E4FEFFB1
:01344D00225C
:102D6A007E137FA91233C9EF4E70037F01227E13AF
:102D7A007FAC1233C9EF4E600C123C4CEF24D024C6
:102D8A00FF920E8002D20E7E137FB21233C9EF4E2B
:102D9A00600C123C4CEF24D0906683F08005E490DE
:102DAA006683F07E137FB81233C9EF4E600C123C73
:102DBA004CEF24D090668DF08005E490668DF07E0D
:102DCA00137FBE1233C9EF4E600C123C4CEF24D075
:102DDA009062B6F08005E49062B6F07E137FC4126A
:102DEA0033C9EF4E600C123C4CEF24D024FF920101
:102DFA008002C20190634163A20190667D63A201D1
:102E0A007F0612235530013B7E137FCA1233C9EF66
:102E1A004E603012000390667DEFF0120003906658
:102E2A007EEFF012000390667FEFF01200039066C7
:102E3A0080EFF0120003906681EFF01200039066B3
:062E4A0082EFF07F002280
:10208700C201E490668DF0D20EC204906683F09090
:1020970062B6F090634163A20190667D63A2017FFF
:1020A70006122355E4F525E52575F003A424D0F59C
:1020B70082E43413F583E493FB740193FA74029377
:1020C700F9121E047003022279E4F526F527FD7440
:1020D7002F2DF582E43461F583E0FF70030222744B
:1020E700E52575F003A424D0F582E43413F583E4E1
:1020F70093FB740193FA740293F985268275830022
:10210700121E1DFEEFB5060875270105260222706F
:10211700E5277003022270EE600302226BE5252497
:10212700FE6028147003022253147003022257140E
:10213700700302225F147003022263240560030206
:10214700227490668D7401F0022274D201742F2DCF
:10215700F582E43461F583E0FF642D700302227495
:10216700123B1DEFC454F0FC74302DF582E434614A
:10217700F583E0FF123B1DEF2C90667DF074312D47
:10218700F582E43461F583E0FF123B1DEFC454F0A0
:10219700FC74322DF582E43461F583E0FF123B1DB8
:1021A700EF2C90667EF074332DF582E43461F5836D
:1021B700E0FF123B1DEFC454F0FC74342DF582E4AC
:1021C7003461F583E0FF123B1DEF2C90667FF074BE
:1021D700352DF582E43461F583E0FF123B1DEFC432
:1021E70054F0FC74362DF582E43461F583E0FF1278
:1021F7003B1DEF2C906680F074372DF582E4346137
:10220700F583E0FF123B1DEFC454F0FC74382DF545
:1022170082E43461F583E0FF123B1DEF2C90668169
:10222700F074392DF582E43461F583E0FF123B1D2C
:10223700EFC454F0FC743A2DF582E43461F583E081
:10224700FF123B1DEF2C906682F08021D204801D87
:102257009066837401F08015C20E80119062B67487
:1022670001F08009E4F527F5260D0220D6052502A1
:0222770020AE97
:012279002242
:103A9200906579E0C3947C503D906579E0FE04F036
:103AA20074B72EF582E43462F583EFF0BF0A2790F3
:103AB2006579E0FF04F074B72FF582E43462F58390
:103AC200E4F0906579E0FF1235D69065797408F0DC
:073AD2009062B8E004F0224D
:103A39009080007480F090633963A201F583F58268
:103A490063A2017F0812235590634163A20190800C
:103A59008863A2017F0A122355908092E4F0A3742F
:103A690032F0A37401F090634BE0FF9080B1F090C5
:103A790080E1EFF09080957455F0A3F09080007488
:093A890001F09080097470F02234
:10374D00908009E04410F09080A0E0706C9080A112
:10375D007482F09080A874FFF0A3F0A3F0A3F07F23
:10376D00039080AEEFF07FCBA3EFF07F039080ACA2
:10377D00EFF0A374CBF09080007402F0906A5C12AD
:10378D001F5500000000906A5CE0908040F0906A48
:10379D005DE0908041F0906A5EE0908042F0906A2A
:1037AD005FE0908043F0A3E4F0A3F0A3F0A3F090CA
:0937BD008018F0A3F0A3F0A3F0C2
:0137C60022E0
:10391900908009E04440F09080D17482F090634C2B
:10392900E0FF9080DEF090634DE0FF9080DFF09043
:1039390080027402F0906A60121F55000000009026
:103949006A60E0908058F0906A61E0908059F09048
:103959006A62E090805AF0906A63E090805BF0A31D
:10396900E4F0A3F0A3F0A3F0908030F0A3F0A3F06B
:02397900A3F0B9
:01397B002229
:1037C700908009E04420F09080B8E0706C9080B958
:1037D7007482F07F039080C6EFF07FCDA3EFF07F78
:1037E700039080C4EFF0A374CDF09080C074FFF015
:1037F700A3F0A3F0A3F09080017402F0906A641222
:103807001F5500000000906A60E090804CF0906ABD
:1038170061E090804DF0906A62E090804EF0906A8F
:1038270063E090804FF0A3E4F0A3F0A3F0A3F0903F
:093837008024F0A3F0A3F0A3F03B
:013840002265
:10344E008C258D26A907EAFDE975F018A424ACFF9A
:10345E00E5F034808F82F583EDF0EBFDE975F01821
:10346E00A4FFAEF024ACFBEE34808B82F583A3ED8B
:10347E00F08526828C83E0FDEF24A8FFEE3480FEDB
:10348E008F82F583EDF08526828C83A3E08F828E6A
:10349E0083A3F0852682852583A3A3E0FDE975F03D
:1034AE0018A424A8FFE5F03480FE8F82F583A3A331
:1034BE00EDF08526828C83A3A3A3E08F828E83A357
:0434CE00A3A3F022A2
:0634D2008D2AAB07AA06DB
:1034D800906A5CE0FCA3E0FDA3E0FEA3E0F52E8E7D
:1034E8002D8D2C8C2BAE02AF038E838F8263A201AD
:1034F800E52D540744C0F583852E8263A201AF2AC7
:103508001223BE908000E020E5F9E4FCFDFEE52EE4
:10351800252AF52EEE352DF52DED352CF52CEC352F
:103528002BF52B908040E52BF0A3E52CF0A3E52D9F
:10353800F0A3E52EF09080007420F0AF2EAE2DADF4
:0B3548002CAC2B906A5C121F49AF2ACC
:013553002255
:0636D2008D25AB07AA06DE
:1036D800906A60E0FCA3E0FDA3E0FEA3E0F5298E7C
:1036E800288D278C26AE02AF038E838F8263A201BA
:1036F800E528540744D0F58385298263A201AF25C4
:103708001223BEE4FCFDFEE5292525F529EE352822
:10371800F528ED3527F527EC3526F526908058E570
:1037280026F0A3E527F0A3E528F0A3E529F090808B
:10373800027420F0AF29AE28AD27AC26906A60123B
:043748001F49AF2541
:01374C00225A
:0230DF008F253B
:1030E100908001E030E5037F0022906A64E0FCA358
:1030F100E0FDA3E0FEA3E0F5298E288D278C269024
:10310100667D63A201E528540744C8F583852982B9
:1031110063A2017F061223D4E5292406F529E435AB
:1031210028F528E43527F527E43526F52690657B33
:1031310063A201E528540744C8F58385298263A267
:1031410001AF251223D4E4FCFDFEE5292525F5294F
:10315100EE3528F528ED3527F527EC3526F52690AF
:10316100804CE526F0A3E527F0A3E528F0A3E529A7
:10317100F09080017420F0AF29AE28AD27AC2690E5
:073181006A64121F49AF252B
:013188002224
:102B63009081E0E0F52505250525052505250525A5
:102B730005250525052505250525908010E0F52863
:102B8300A3E0F529A3E0F52AA3E0F52B9081E1E08A
:102B9300F5250525052505250525052505250525F2
:102BA300052505250525908014E0F52CA3E0F52DDA
:102BB300A3E0F52EA3E0F52FE52EB52A08E52FB502
:102BC3002B037F0022E4F525E52E540744E0F5832B
:102BD300852F8263A20190637863A2017F08122389
:102BE300EC90637A63A2019062B063A2017F061244
:102BF3002355906378E0F526A3E0F527E4F52590C7
:102C03006378E0702AA3E024F8F525E52E54074401
:102C1300E0F583852F8274082582F582E43583F5F8
:102C23008363A20190637863A201AF251223ECAE04
:102C330026E4FCFDE52F2527F52FE52E3EF52EEDA9
:102C4300352DF52DEC352CF52C908014E52CF0A3C7
:102C5300E52DF0A3E52EF0A3E52FF090800074405E
:032C6300F0AF25AA
:012C6600224B
:10277B009081E6E0F525052505250525052505258B
:10278B0005250525052505250525908028E0F52837
:10279B00A3E0F529A3E0F52AA3E0F52B9081E7E070
:1027AB00F5250525052505250525052505250525DE
:1027BB0005250525052590802CE0F52CA3E0F52DAE
:1027CB00A3E0F52EA3E0F52FE4F525E52EB52A0AB7
:1027DB00E52FB52B05C2080228D5E52E540744F08A
:1027EB00F583852F8263A20190637863A2017F0832
:1027FB001223EC906378E0F526A3E0F527E5274557
:10280B002670099080027410F07F0022906684E09D
:10281B00FFF4602D90637AE06F7076906685E0FF31
:10282B0090637BE06F706A906686E0FF90637CE05C
:10283B006F705E906687E0FF90637DE06F60228033
:10284B005090637AE0906684F090637BE0906685AD
:10285B00F090637CE0906686F090637DE0906687F5
:10286B00F0906378E0702AA3E024F8F525E52E5468
:10287B000744F0F583852F8274082582F582E435B1
:10288B0083F58363A20190637863A201AF251223C2
:10289B00ECAE26E4FCFDE52F2527F52FE52E3EF5C6
:1028AB002EED352DF52DEC352CF52CAF2BAE2AADB1
:1028BB0029AC28AB2FAA2EA92DA82CD3121F384038
:1028CB00099080027410F07F002290802CE52CF090
:1028DB00A3E52DF0A3E52EF0A3E52FF09080027475
:0428EB0040F0AF25E5
:0128EF0022C6
:1028F0009081E3E0F5250525052505250525052518
:102900000525052505250525052590801CE0F528CC
:10291000A3E0F529A3E0F52AA3E0F52B9081E4E0FC
:10292000F525052505250525052505250525052567
:10293000052505250525908020E0F52CA3E0F52D43
:10294000A3E0F52EA3E0F52FE4F525E52EB52A0A40
:10295000E52FB52B05C209022A3BE52E540744E8B2
:10296000F583852F8263A20190600463A2017F0E2C
:10297000122402906004E0F526A3E0F52790600C95
:10298000E0FFF4604590667DE0FEEF6E706EA3E0C0
:10299000FF90600DE06F706490667FE0FF90600EC6
:1029A000E06F7058906680E0FF90600FE06F704CB1
:1029B000906681E0FF906010E06F7040906682E06A
:1029C000FF906011E06F60048032D2D9906004E023
:1029D000702AA3E024F2F525E52E540744E8F58398
:1029E000852F82740E2582F582E43583F58363A2F8
:1029F0000190600463A201AF25122402AE26E4FC1C
:102A0000FDE52F2527F52FE52E3EF52EED352DF58D
:102A10002DEC352CF52CAF2BAE2AAD29AC28AB2FE5
:102A2000AA2EA92DA82CD3121F385006E52745261B
:102A300070099080017410F07F0022908020E52CB6
:102A4000F0A3E52DF0A3E52EF0A3E52FF090800193
:052A50007440F0AF2509
:012A5500225E
:042E50008E2A8F2B0C
:102E5400906A5CE0FCA3E0FDA3E0FEA3E0F5318E04
:102E6400308D2F8C2EE531FFE5305407FEE42FF52D
:102E74002DEE34C0F52C852D82F5837423F0052DB9
:102E8400E52D7002052C532CC7F582852C83740A1A
:102E9400F0052DE52D7002052C532CC7906341637A
:102EA400A201852C83852D8263A2017F061223BE95
:102EB4007406252DF52DE4352CF52C852A83852BD8
:102EC4008263A201852C83852D8263A2011223A231
:102ED400908000E020E5F9E4FCFDFE906A5CE0F8F7
:102EE400A3E0F9A3E0FAA3E02FFFEE3AFEED39FDEB
:102EF400EC38FCEF2408FFE43EFEE43DFDE43CFC3A
:102F0400906A5C121F49906A5CE0908040F0906A7D
:102F14005DE0908041F0906A5EE0908042F0906ABB
:0C2F24005FE0908043F09080007420F08B
:012F3000227E
:06300B008E2A8F2B8D2C94
:10301100906A5CE0FCA3E0FDA3E0FEA3E0F5328E44
:10302100318D308C2FE532FFE5315407FEE42FF569
:103031002EEE34C0F52D852E82F5837423F0052EF6
:10304100E52E7002052D532DC7F582852D83EBF0FA
:10305100052EE52E7002052D532DC790634163A205
:1030610001852D83852E8263A2017F061223BE7402
:1030710006252EF52EE4352DF52D852A83852B8207
:1030810063A201852D83852E8263A201AF2C1223B9
:10309100BE908000E020E5F97408252CF52CFFE4B2
:1030A100FCFDFEE5322FF532EE3531F531ED3530EF
:1030B100F530EC352FF52F908040E52FF0A3E5306A
:1030C100F0A3E531F0A3E532F09080007420F0AF79
:0D30D10032AE31AD30AC2F906A5C121F4959
:0130DE0022CF
:0235D6008F3F25
:1035D800906A5CE0FCA3E0FDA3E0FEA3E0F5438E67
:1035E800428D418C40E543FFE5425407FEE42FFF3E
:1035F800EE34C09062B763A201F5838F8263A201A3
:10360800AF3F1223BE908000E020E5F9E4FCFDFE08
:10361800E543253FF543EE3542F542ED3541F541A9
:10362800EC3540F540908040E540F0A3E541F0A33B
:10363800E542F0A3E543F09080007420F0AF43AE7C
:0B36480042AD41AC40906A5C121F498B
:013653002254
:062F31008E2A8F2BAB0578
:102F3700906A5CE0FCA3E0FDA3E0FEA3E0F5318E20
:102F4700308D2F8C2EE531FFE5305407FEE42FF549
:102F57002DEE34C0F52C852D82F5837423F0052DD5
:102F6700E52D7002052C532CC7F582852C83EBF0D9
:102F7700052DE52D7002052C90634163A201852C78
:102F870083852D8263A2017F061223BE7406252D39
:102F9700F52DE4352CF52C532CC7E52A852D828594
:102FA7002C83F0052DE52D7002052C532CC7F582D7
:102FB700852C83E52BF0052DE52D7002052C532C70
:102FC700C7908000E020E5F9E531240AF531E435C2
:102FD70030F530E4352FF52FE4352EF52E9080406F
:102FE700E52EF0A3E52FF0A3E530F0A3E531F0904F
:102FF70080007420F0AF31AE30AD2FAC2E906A5CFC
:03300700121F494C
:01300A0022A3
:103C3000E5D220E0FBC2AF438E2075D2028F828E88
:0B3C400083E0FFE4F5D2538EDFD2AF2B
:013C4B002256
:103C6600E5D220E0FBC2AF43D2028F828E83EDF015
:093C760075D25063D250D2AF2286
:10365400E4FDED2401FFE433FE123C3074392DF512
:1036640082E43463F583EFF00DBD3FE6E4FDED2421
:103674007FFFE433FE123C30742F2DF582E4346175
:10368400F583EFF0742F2DF582E43461F583E07057
:103694001B742F2DF582E43461F5837420F07430AB
:1036A4002DF582E43461F583E4F080040DBD80BE21
:1036B400E49061AEF0FDEDFF7E00123C3074AF2D5E
:0D36C400F582E43461F583EFF00DBDFEE901
:0136D10022D6
:023B55008B2AB9
:103B5700A2AF920FC2AF85A22B53A2FE8E838F8294
:103B670005A28C838D82740912241AE52A53A2FEBA
:103B770043A22012241C53A2DF852BA2A20F92AFCF
:013B8700FF3E
:013B8800221A
:103BF700A2AF920FC2AF8C838D82EF12241A43A219
:0C3C07002012241C53A2DFA20F92AFFF7A
:013C1300228E
:023BAF008F2560
:103BB100A2AF920FC2AFE4F5838D82740612241A6C
:103BC100E52543A22012241C53A2DFA20F92AF7F4E
:013BD10001F2
:013BD20022D0
:023BD3008F253C
:103BD500A2AF920FC2AFE4F5838D82740A12241A44
:103BE500E52543A22012241C53A2DFA20F92AF7F2A
:013BF50001CE
:013BF60022AC
:10227A00A907E7FFA805EF93C3966008403B74FCE3
:10228A002FFF80F00F08EF93C3966008402B74FB72
:10229A002FFF80E00F08EF93C3966008401B74FA83
:1022AA002FFF80D00F08EF93D3966008400B74F984
:1022BA002FFF80C01F1F1F1F1FEF54FEF80303F7D5
:1022CA00E893FC08E893FD08E893FE08E893FF22E8
:1022DA0009E993C39D6008402974FB29F980F10933
:1022EA00E993C39E6008401A74FA29F980E209E961
:1022FA0093D39F6008400B74F929F980D3191919EF
:10230A001919E9C313C313FF22740093F8ECC39895
:10231A004024701F740193F8EDC398401970147427
:0E232A000293F8EEC398400E7009740393F806
:10233800EFC39840037F00227F0122EDF8E6F00802
:10234800A3DFFA22EDF8E0F608A3DFFA22E0A363A0
:10235800A201F0A363A201DFF475A20022E0A36347
:10236800A201F0A363A201E0A363A201F0A363A208
:1023780001E463A201F0A363A201DFE175A20022D8
:10238800E0A363A2016DFE936CFDEE058393FC153B
:102398008363A201DFEA75A200227F00E493A363AE
:1023A800A201F00F600CA3E583C2E3F58363A201E9
:1023B80080EA75A20022E0A363A201F0A3E583C22C
:1023C800E3F58363A201DFEE75A20022E0A363A216
:1023D80001F0A3E583C2E4D2E3F58363A201DFEC55
:1023E80075A20022E583C2E3F583E0A363A201F0AE
:1023F800A363A201DFEE75A20022E583C2E4D2E363
:10240800F583E0A363A201F0A363A201DFEC75A248
:102418000022F922C002C004C00612FFF0D006D084
:0424280004D00222B8
:1013E8003E2A2C312CCFE0F0E0ECE5F2F0FB20F8BF
:1013F800E8EDFB2043414E0A003E4C2C6B30312C6B
:1014080025732C43EAEEF0EEF1F2FC20EDE020F833
:10141800E8EDE52043414E2C30202D20353030EAD0
:10142800E1283530EC292C31202D203530EAE1280F
:10143800353030EC290A0030202D20353030EAE1F3
:10144800283530EC290031202D203530EAE12835C7
:101458003030EC29003E2A2C312CCFE0F0E0ECE5CE
:10146800F2F0FB20EFF0EEF2EEEAEEEBE0204D4F6B
:10147800444255530A003E4C2C4930312C256C759A
:101488002CD1EAEEF0EEF1F2FC20EEE1ECE5EDE035
:101498002C343830302C393630302C313932303029
:1014A8000A003E532C4931322C2562752CC0E4F0D9
:1014B800E5F120E1EBEEEAE020D2C8D220EDE02011
:1014C800F8E8EDE50A003E532C6D2562752C25627F
:1014D800752D25752D2562752D2562752CCFF0E8A3
:1014E800E1EEF0202562752028B9CFF02DD0E5E394
:1014F8002DCAEEEB2DD2E8EF290A003E532C5630C8
:10150800382C2562752CC8EDF2E5F0E2E0EB20EE10
:10151800EFF0EEF1E0282A3130ECF1290A003C2105
:10152800003C6B30313D003C4930313D003C493195
:10153800323D003C5630383D002043616E457247CD
:10154800495400200A002043616E457272434821C5
:10155800000A00CFF0E8E5EC3A00CEF8E8E1EAE06E
:1015680020CAD1210A00CED8C8C1CAC021000AC7E2
:10157800E0EFF0EEF13A003C6D303D000000003C39
:101588006D313D000000003C6D323D000000003C24
:101598006D333D000000003C6D343D000000003C10
:1015A8006D353D000000003C6D363D000000003CFC
:1015B8006D373D000000003C6D383D000000003CE8
:1015C8006D393D000000003C6D31303D0000003CAD
:1015D8006D31313D0000003C6D31323D0000003C72
:1015E8006D31333D0000003C6D31343D0000003C5E
:1015F8006D31353D00000000C1814001C0804101CE
:10160800C0804100C1814001C0804100C1814000CB
:10161800C1814001C0804101C0804100C1814000BA
:10162800C1814001C0804100C1814001C0804101A9
:10163800C0804100C1814001C0804100C18140009B
:10164800C1814001C0804100C1814001C080410189
:10165800C0804100C1814000C1814001C08041017A
:10166800C0804100C1814001C0804100C18140006B
:10167800C1814001C0804101C0804100C18140005A
:10168800C1814001C0804100C1814001C080410149
:10169800C0804100C1814000C1814001C08041013A
:1016A800C0804100C1814001C0804100C18140002B
:1016B800C1814001C0804100C1814001C080410119
:1016C800C0804100C1814001C0804100C18140000B
:1016D800C1814001C0804101C0804100C1814000FA
:1016E800C1814001C0804100C1814001C0804101E9
:1016F800C0804100C1814000C0C101C30302C2C60D
:101708000607C705C5C404CC0C0DCD0FCFCE0E0AF5
:10171800CACB0BC90908C8D81819D91BDBDA1A1E95
:10172800DEDF1FDD1D1CDC14D4D515D71716D6D265
:101738001213D311D1D010F03031F133F3F2323625
:10174800F6F737F53534F43CFCFD3DFF3F3EFEFA35
:101758003A3BFB39F9F83828E8E929EB2B2AEAEE75
:101768002E2FEF2DEDEC2CE42425E527E7E62622A5
:10177800E2E323E12120E0A06061A163A3A2626605
:10178800A6A767A56564A46CACAD6DAF6F6EAEAA75
:101798006A6BAB69A9A86878B8B979BB7B7ABABE15
:1017A8007E7FBF7DBDBC7CB47475B577B7B67672E5
:1017B800B2B373B17170B0509091519353529296E5
:1017C800565797559594549C5C5D9D5F9F9E5E5AB5
:1017D8009A9B5B99595898884849894B8B8A4A4EF5
:1017E8008E8F4F8D4D4C8C44848545874746868225
:0717F8004243834181804060
:103C1A0052668F0000000000000000000000000053
:053C2A00000000000095
:013C9600220B
:030023000238415F
:10384100C0E0C083C082C0D075D01830982CE55C30
:1038510025E9F5EB30D709E55B25F904F5FB800691
:10386100E55B25F9F5FBD29174382556F582E434F0
:1038710069F583E599F00556C298309929E559C350
:1038810095555013AF59055974382FF582E4346AB0
:10389100F583E0F599800DAF558F59EF6006055915
:0F38A100D296C290C299D0D0D082D083D0E032DC
:103B8900C2A9438902758C48758A4875D90475DBC1
:103B99004875DC4875DD4875DE48E4F5E9F5F9C294
:063BA900D9D28CD2DE220D
:102C67007BFF7A1379E81218619068A1E0701475F8
:102C77002EFF752F1475303F7BFF7A1479011218D8
:102C8700618012752EFF752F1475304E7BFF7A14F5
:102C970079011218617BFF7A14795D121861906AC5
:102CA7005AE0FEA3E0FFC3E49FFFE49EFEAB07FAF2
:102CB7003395E0F9F87F007E8C7D0A7C00121E9820
:102CC7008F318E308D2F8C2E7BFF7A14797E1218E0
:102CD700617BFF7A1479AA9068A2E0F52E12186139
:102CE700E4F52A7BFF7A1479CE852A2EE52AFD336F
:102CF70095E0FC74A52DF58274683CF583E0F52F0B
:102D0700AF2AEF3395E0FEEF25E0FFEE33FE74B612
:102D17002FF58274683EF583E0F530A3E0F5317452
:102D2700D62DF58274683CF583E0F532AF2AEF3390
:102D370095E0FE74E72FF58274683EF583E0F5337E
:102D4700E52A04F534121861052AC3E52A6480943C
:102D57009040907BFF7A157903906A59E0F52E121F
:022D67001861F1
:012D69002247
:10242C007E157F261233C9EF4E70037F0122E49094
:10243C0068A1F07E157F291233C9EF4E601B123C48
:10244C004C8F25E525B431069068A1740AF0E5257A
:10245C00B432069068A17464F07E157F2F1233C9D4
:10246C00EF4E60231239DCA804A905AA06AB077F3E
:10247C00007E8C7D0A7C00121E98121F2A906A5ACC
:10248C00EEF0A3EFF0800A906A5A74FFF0A374B8D0
:10249C00F07E157F351233C9EF4E600A1239DC908D
:1024AC0068A2EFF08005E49068A2F07E157F3B12E5
:1024BC0033C9EF4E600D1239DC906A58EEF0A3EF81
:1024CC00F08009906A58E4F0A37464F0906A58E0C4
:1024DC00FEA3E0FF7C007D64121E4A8E5B8F5CE4E1
:1024EC00F525AF25EF3395E0FEEF7803C333CE33FC
:1024FC00CED8F9247FF58274153EAF82FE1233C913
:10250C00EF4E60681239DCE525FD3395E0FC74A5CF
:10251C002DF58274683CF583EFF01239DCAD07AC15
:10252C0006AF25EF3395E0FEEF25E0FFEE33FE74AA
:10253C00B62FF58274683EF583ECF0A3EDF01239FA
:10254C00DCE525FD3395E0FC74D62DF58274683CF2
:10255C00F583EFF01239DCE525FD3395E0FC74E7EB
:10256C002DF58274683CF583EFF0804EE525FD3344
:10257C0095E0FC74A52DF58274683CF583E4F0AF0E
:10258C0025EF3395E0FEEF25E0FFEE33FE74B62F1A
:10259C00F58274683EF583E4F0A3F074D62DF582D1
:1025AC0074683CF583E4F0AF25EF3395E0FE74E7F7
:1025BC002FF58274683EF583E4F00525C3E52564A8
:0A25CC0080949050030224EE7F007B
:0125D60022E2
:1038B00043AB01C2E8C2EAE4FFEFC454F0F5B1C380
:1038C000EF64809488500575B3D08003E4F5B3E4C9
:1038D000F5B275BCC8F5BDF5BE75BF7875C4FFF50A
:1038E000C5F5C675C778F5A3F5A3F5A3F5A3F5A3AC
:1038F000F5A3F5A3F5A30FBF0EBF9068A1E0FF25C8
:10390000E0F5B475B50C75B66C75A11275AB0275A2
:08391000C13E75C3FF75C2033F
:01391800228C
:10397C0075B180E4F5B3F5B28545BCE5465403FF5B
:10398C0033333354F8FFE54654E04FFFE547C41397
:10399C0054074FF5BDE54733333354F8FFE548C4BE
:1039AC001354074FF5BEE54833333354F8F5BF8550
:1039BC004AA3854BA3854CA3854DA3854EA3854F68
:1039CC00A38550A38551A3E549540F2450F5B32288
:102A5600E59B541F6020200A1A7E157F41122E50D6
:102A6600E59B541FFF7E007D03122F317E157F4BA1
:102A7600122E50E4F59BE5BA30E008E4F5B375B1E3
:102A860080F5B2E5CFF47003022B60752901E4F5F9
:102A960028E5CFF455297003022B4EE528C454F0DF
:102AA600F5B1E5B2547F6420706FE5B3540FF54974
:102AB60085BC45E5BD541FFF131313541FFFE5BD29
:102AC60054E044184FF546E5BDC43354E0FFE5BE77
:102AD600131313541F4FF547E5BEC43354E0FFE507
:102AE600BF131313541F4FF54885A34A85A34B857F
:102AF600A34C85A34D85A34E85A34F85A35085A3DF
:102B060051E4F5B2E545547EB5450575B3508003ED
:102B160075B3D0E5492405FF22E5B2549F60232012
:102B26000A207E157F4E122E50AFB27E007D031214
:102B36002F31AFB37E007D03122F317E157F5912E0
:102B46002E50E4F5B275B3D0E52925E0F529052820
:0C2B5600E528C394085003022A977F0072
:012B62002250
:10355400C218E4F556F50BD296C219F554F555F593
:1035640059FF7F409068F8E4F0A3DFFC7F40E4F566
:1035740057F558F55AF55E12242C1238B0C2ADE452
:10358400F5C9D2CDD2CCC2C9C2CAF5CDF5CC906AA8
:103594005AE0F5CBA3E0F5CA85CBCD85CACCE4F5DA
:1035A40098D29E438740C29FC2ACC298C29975B854
:1035B4001075B710D2CAD29CD2AC123B89C2D9E5DD
:1035C400E92464F5EB30D706E5F904F5FB2285F927
:0135D400FBFB
:0135D50022D3
:013C9700220A
:013C98002209
:05001E00D29CD2AC22CF
:013C99002208
:063AD900AC05AB07AA06D4
:103ADF009068E674FFF09068F7F0AF041CEF602D6C
:103AEF000BEBAE0270010A14F5828E83E0FF906833
:103AFF00E6E06FFF9015FF93FE9068F7E06E906819
:0D3B0F00E6F0EF9016FF939068F7F080CD80
:013B1C002286
:10333F0074E72554F582E43468F583E07006F5549C
:10334F00F557F55874A52554F582E43468F583E0F4
:10335F00906A38F074E72554F582E43468F583E019
:10336F00906A39F0E55425E024B6F582E43468F527
:10337F0083E0FCA3E0FDEC906A3AF0A3EDF0E4A348
:10338F00F074D62554F582E43468F583E0906A3DF5
:10339F00F07E6A7F387D06123AD99068E6E0906A2F
:1033AF003EF09068F7E0906A3FF0E4F559755508E4
:0A33BF00C296C2992099FDD299220E
:10322500E55EC394404003E4F55E74F8255EF582DF
:10323500E43468F583E0FF30E16F74F8255EF582CC
:10324500E43468F583EF54FDF0E4906478F0A374FA
:103255000DF090667CE090647AF0A37419F0A37485
:1032650048F0A37479F0E55E131313541FFF9068BB
:10327500A2E02F90647EF0E55E540725E025E0246A
:1032850080A3F0A37408F0F5F0E55EA424A1F5820F
:10329500E5F03466F58363A20190648163A2017F42
:0E32A50008122355055E7F0122055E7F002280
:013C9A002207
:101B5B0074F8255AF582E43468F583E020E0020539
:101B6B005AE55AC394404003E4F55A122A56EF60E3
:101B7B0069E548640F70639068A2E0FF6547705A8F
:101B8B0074F8255AF582E43468F583E0FE30E04AB8
:101B9B0074F8255AF582E43468F583EE54FEF0753B
:101BAB004548754679E55A131313541FFEEF2EF56E
:101BBB0047E55A540725E025E02480F54875490888
:101BCB0075F008E55AA424A1F582E5F03466F58397
:101BDB007D4A7F0812234C12397C300249C2029095
:101BEB0068A4E004F070069068A3E004F0D390685A
:101BFB00A4E094B89068A3E0940B402AE4F0A3F01F
:101C0B00F52574F82525F582E43468F583E030E298
:101C1B000E74F82525F582E43468F5837403F0051A
:101C2B0025E525B440DC20D903021E03C2D9E556B5
:101C3B00D394005003021DAEC29185565DE4F55658
:101C4B008557268558277E697F3890693AE02405A9
:101C5B00FD123AD9200A127E157F5B122E507E6937
:101C6B007F38E4FBAD5D12300B9068F7E0FF9068B6
:101C7B00E6E04F6010300A03021DAE7E157F621244
:101C8B002E50021DAE74A52554F582E43468F583FD
:101C9B00E0FF906938E0B5071474E72554F582E44A
:101CAB003468F583E0FF906939E06F6010300A0308
:101CBB00021DAE7E157F6E122E50021DAEE4F52571
:101CCB0090693AE0FFE525C39F4003021DAE74A166
:101CDB002527F58274663526F583E0FF743C2525B0
:101CEB00F582E43469F583E0FEEF6E602774A1257D
:101CFB0027F58274663526F583EEF0E527AE267858
:101D0B0003CEC313CE13D8F924F8F58274683EF5CD
:101D1B00837407F0E527AE267803CEC313CE13D812
:101D2B00F924F8F58274683EF583E04404F0052746
:101D3B00E5277002052624A1F58274663526F58306
:101D4B00E0FF743B2525F582E43469F583E0FEEF73
:101D5B006E602774A12527F58274663526F583EE10
:101D6B00F0E527AE267803CEC313CE13D8F924F8AB
:101D7B00F58274683EF5837407F0E527AE26780389
:101D8B00CEC313CE13D8F924F8F58274683EF583CD
:101D9B00E04404F00527E5277002052605250525F7
:101DAB00021CCBE555601974D62554F582E43468D2
:101DBB00F583E02558F558E43557F557055480075A
:101DCB00E4F554F557F558D29012333FE5E924E882
:101DDB00F5EB30D708E5F92404F5FB8006E5F9248B
:101DEB0003F5FB200A127E157F76122E507E6A7F3A
:081DFB0038E4FB7D0812300BF7
:011E030022BC
:033C93007F00228D
:1032BF00020881E493A3F8E493A34003F68001F29C
:1032CF0008DFF48029E493A3F85407240CC8C33310
:1032DF00C4540F4420C8834004F456800146F6DFDF
:1032EF00E4800B0102040810204080903C14E47E1F
:1032FF00019360BCA3FF543F30E509541FFEE493D4
:10330F00A360010ECF54C025E060A840B8E493A39A
:10331F00FAE493A3F8E493A3C8C582C8CAC583CAC5
:10332F00F0A3C8C582C8CAC583CADFE9DEE780BE7D
:013C2F000094
:101E0400BB010689828A83E0225002E722BBFE02DC
:091E1400E32289828A83E493220F
:101E1D00BB010CE58229F582E5833AF583E022507A
:101E2D0006E92582F8E622BBFE06E92582F8E222C4
:0D1E3D00E58229F582E5833AF583E49322DE
:101E4A00EF8DF0A4A8F0CF8CF0A428CE8DF0A42EAC
:021E5A00FE2266
:101E5C0075F008758200EF2FFFEE33FECD33CDCC3D
:101E6C0033CCC58233C5829BED9AEC99E5829840C0
:101E7C000CF582EE9BFEED9AFDEC99FC0FD5F0D69D
:101E8C00E4CEFBE4CDFAE4CCF9A88222B800C1B9C7
:101E9C000059BA002DEC8BF084CFCECDFCE5F0CB05
:101EAC00F97818EF2FFFEE33FEED33FDEC33FCEB3E
:101EBC0033FB10D703994004EB99FB0FD8E5E4F9F9
:101ECC00FA227818EF2FFFEE33FEED33FDEC33FCE6
:101EDC00C933C910D7059BE99A4007EC9BFCE99ADA
:101EEC00F90FD8E0E4C9FAE4CCFB2275F010EF2F1F
:101EFC00FFEE33FEED33FDCC33CCC833C810D7071F
:101F0C009BEC9AE899400AED9BFDEC9AFCE899F859
:0E1F1C000FD5F0DAE4CDFBE4CCFAE4C8F922EC
:0E1F2A00C3E49FFFE49EFEE49DFDE49CFC22C8
:101F3800EB9FF5F0EA9E42F0E99D42F0E89C45F0FF
:011F48002276
:0C1F4900ECF0A3EDF0A3EEF0A3EFF0220B
:101F5500A8828583F0D083D082121F6C121F6C1269
:101F65001F6C121F6CE473E493A3C583C5F0C5838E
:101F7500C8C582C8F0A3C583C5F0C583C8C582C8D6
:011F85002239
:1017FF00E53A242EF8E6053A22782B301602782E99
:10180F00E475F001121FE7021E04200FEB7F2ED2AA
:10181F000F8018EF540F2490D43440D4FF30130BA3
:10182F00EF24BFB41A0050032461FFE53B6002159B
:10183F003B053EE53E7002053D30160D782BE475F5
:10184F00F001121FE7EF021F86023A927403D216BD
:10185F008003E4C216F53A8B2B8A2C892DE4F53BD5
:10186F00F53DF53EE53B60077F2012183A80F57590
:10187F003CFFC210C20FC211C212C214C215C2174E
:10188F00121808FF700D3016057F0012184BAF3E6F
:10189F00AE3D22B4255FC2D5C213121808FF24D063
:1018AF00B40A00501A75F00A783B30D50508B6FF18
:1018BF000106C6A426F620D5047002D21280D924C0
:1018CF00CFB41A00EF5004C2E5D213021A4BD21054
:1018DF0080C6D20F80C0D21180BCD2D580BAD214AC
:1018EF0080B47F2012183A2011077401B53B0040D5
:1018FF00F11217FFFF12183A021873D217D2158080
:10190F00951217FFFB1217FFFA1217FFF94A4B70C8
:10191F0006791C7A1B7BFF20112EE53B602A7E0087
:10192F008E82758300121E1D60060EEE653C70F0F0
:10193F00C2D5EBC0E0EAC0E0E9C0E0EE121A92D0E7
:10194F00E0F9D0E0FAD0E0FB121E04FF60AAEBC072
:10195F00E0EAC0E0E9C0E012183AD0E02401F9D083
:10196F00E03400FAD0E0FBE53C0460DCD53CD980E4
:10197F00877BFF7A1A798ED211809C791080027939
:10198F0008C215C2178008D2D5790A8004790AC215
:10199F00D5E53C047002F53CE4FAFDFEFF1217FF9B
:1019AF00FC7B082010131217FFFD7B10300F0A125B
:1019BF0017FFFE1217FFFF7B20EC3382D592D55015
:1019CF0013C3E4300F069FFFE49EFEE42010039D37
:1019DF00FDE49CFCE4CBF8C210EC700CCFCECDCC68
:1019EF00E824F8F870F38017C3EF33FFEE33FEED02
:1019FF0033FDEC33FCEB33FB994002FB0FD8E9EBE3
:101A0F00301005F8D0E0C448B210C0E00AEC4D4EDB
:101A1F004F78207B0070C2EAB53C0040BCC0E0129A
:101A2F001A94D0F0D0E0201004C4C0E0C4B210C0AB
:101A3F00F0121823D0F0D5F0EB02187312204619CC
:101A4F001053198A5818E14C18DD42198E4F199608
:0F1A5F004419964918F643199C55198046198069
:101A6E00451980471B3C5018E52D18E92E190C2BF3
:101A7E0018ED23190A201B252A18A5480000190461
:101A8E003F3F3F00790AA2D5201214301409B91035
:101A9E00020404B9080104A2D52015025001042045
:101AAE0011689211B53B005034C0E07F20301219FE
:101ABE007F30A21172157214500F121AEBC211C29E
:101ACE0015C214C2177F30800F301403E9C0E01224
:101ADE00183A301403D0E0F9D0E0B53BCC301417EF
:101AEE007F30B9100C12183A7F583013077F788068
:101AFE0003B9080312183A3011057F2D02183A7FE8
:101B0E00202017F87F2B2015F322921180CF286EFC
:101B1E00756C6C2900D2101217FF3010F8C21078B5
:101B2E003B30D50108F60218A52D5043495812171F
:101B3E00FF2403B405004001E4901B379312182BC9
:0D1B4E00743A12182BD212753B0402198A4A
:1025D7008B2A8A2B892CE4F536F535F534F533F556
:1025E70031F532E52E452F452D6012EBC0E0EAC0EC
:1025F700E0E9C0E0AB2DAA2EA92F121FF7AB2A05E1
:102607002CE52CAA2B7002052B14F9121E04F537A2
:10261700C394094007E537D3940D40E1E5376420BB
:1026270060DBE537B42D054332038016E537B42B5D
:1026370005433201800C74FF252CF52C74FF352BD4
:10264700F52BE53060046410703FAB2AAA2BA92C48
:10265700121E0464306009E530702E75300A802937
:10266700900001121E1DFF64786004EFB4581343F5
:1026770032017530107402252CF52CE4352BF52B1F
:102687008007E5307003753008AB2A052CE52CAAC6
:102697002B7002052B14F9121E04F537C394614001
:1026A7000AE537D3947A50035337DF74D02537F5CB
:1026B70037C3940A400CE5379411406D74F92537F8
:1026C700F537E537D39530506043320185363B8582
:1026D700353A853439853338AF307E00E4FCFDABBD
:1026E70036AA35A934A833121F98C8ECC8C9EDC952
:1026F700CAEECACBEFCBE4FCFDFEEB2537F536EE91
:102707003AF535ED39F534EC38F533AF36AE35AD4E
:1027170034FCAB3BAA3AA939A838D3121F38500367
:10272700022690433204022690E53220E003E4803B
:102737002DE52E452F452D601EAB2AE52C24FFF9EC
:10274700E52B34FFFAEBC0E0EAC0E0E9C0E0AB2DCF
:10275700AA2EA92F121FF7E53230E20774FFFFFEFA
:10276700FDFC22E532AF36AE35AD34AC3330E10394
:04277700021F2A22F1
:101F8600BB010689828A83F0225002F722BBFE013A
:021F9600F32234
:101F9800E88FF0A4CC8BF0A42CFCE98EF0A42CFCE8
:101FA8008AF0EDA42CFCEA8EF0A4CDA8F08BF0A466
:101FB8002DCC3825F0FDE98FF0A42CCD35F0FCEBC5
:101FC8008EF0A4FEA9F0EB8FF0A4CFC5F02ECD398A
:0F1FD800FEE43CFCEAA42DCE35F0FDE43CFC22F7
:101FE700FAE6FB0808E6F925F0F618E6CA3AF622FB
:101FF700BB011A89828A83D0F0D0E0F8D0E0F9D00B
:10200700E0FAD0E0FBE8C0E0C0F00220755016E926
:10201700F8D083D082D0E0F9D0E0FAD0E0FBC082DC
:10202700C08302206CBBFE16E9F8D083D082D0E0D3
:0F203700F9D0E0FAD0E0FBC082C08302207E2205
:10204600D083D082F8E4937012740193700DA3A329
:1020560093F8740193F5828883E47374029368603D
:06206600EFA3A3A380DF3D
:09206C00EBF608EAF608E9F62299
:09207500EBF0A3EAF0A3E9F0226C
:09207E00EBF208EAF208E9F22293
:00000001FF
